:040000008A016728E2
:080008000B110900702A7E2A89
:10001000892AB92AEC2A032B3F2B5C2B712B782BD6
:10002000942B112C3B2C752CD52CEB2C3D2D542DC9
:10003000632D772D7E2D8D2DF30000308A00253025
:10004000730703188A0A7308820705308A00B62DE1
:1000500005308A00C42D05308A00D22D05308A0073
:10006000E02D05308A00EE2D05308A00FC2D06308B
:100070008A000A2E06308A00182E06308A00312E99
:1000800006308A004A2E06308A00552E06308A0035
:100090006E2E06308A00AF2E06308A00B92E06304A
:1000A0008A00C72E06308A00D52E06308A00E32E3D
:1000B00006308A00F12E06308A00FF2E07308A00B3
:1000C0000D2F07308A001B2F07308A00252F0330A1
:1000D00083120313850001308600F03083168500FB
:1000E00086019B0180309F00283081008312BC0173
:1000F0003830BD000A203230FD0014208312031373
:10010000BC013830BD000A200A30FD0014208312E3
:100110000313BC013830BD000A200A30FD00142052
:1001200083120313BC010C30BD000A20BC01063051
:10013000BD000A20BC018030BD000A201530FB0044
:100140000F2083120313BC01C030BD000A201830F9
:10015000FB000F200130FF0017201820AC000D20FD
:100160001820B3000D201820AD000D201820B40079
:100170000D201820AE000D201820B5000D201820ED
:10018000AF000D201820B0000D201820B6000D2063
:100190001820B1000D201820B7000D201820B20043
:1001A0000D201820B8000D201B30FC0016208312F3
:1001B00003132C08F000700EF039F039AC0033084E
:1001C0000F39B300F0012C0833070318F00AAC0014
:1001D0002D08F000700EF039F039AD0034080F39F9
:1001E000B400F0012D0834070318F00AAD002E0802
:1001F000F000700EF039F039AE0035080F39B50057
:10020000F0012E0835070318F00AAE002F08073951
:10021000AF003008F000700EF039F039B000360849
:100220000F39B600F001300836070318F00AB000A5
:100230003108F000700EF039F039B10037080F398D
:10024000B700F001310837070318F00AB10032088F
:10025000F000700EF039F039B20038080F39B800EC
:10026000F001320838070318F00AB2001220831296
:100270000313A001A101A201A301A401A501013062
:10028000FD0014201120102083120313810132304D
:10029000FD0014208312031301085A3C0130031897
:1002A0000301FF3903195D29783001020130031879
:1002B0000301FF3903195D290130003C03197F292F
:1002C000112013200108C1000530FD001420831205
:1002D00003130108410203197A291120102001306B
:1002E000FF001720831203130108C1000530FD0031
:1002F0001420672911201320A40A0319A50A050850
:100300002039003C031D6F2A2508A7002408A600F9
:100310000230FF0017208312031305082039003C28
:10032000031D6F2A1E30FC0016202130FC00162011
:10033000831203132508003C0130031CA729003059
:10034000031DA7292408003C013003180301003CC9
:100350000319692AC001023040020318232A15201C
:10036000C008031DB8297908C3007808C200BC2959
:100370007908C5007808C4007408BF000C20243038
:10038000FC001620750883120313BF000C202430D4
:10039000FC001620770883120313BF000C20760898
:1003A000F0007008003C031DD9292730FC001620FE
:1003B000092A7008013C031DE1292A30FC0016209F
:1003C000092A7008023C031DE9292D30FC00162083
:1003D000092A7008033C031DF1293030FC00162067
:1003E000092A7008043C031DF9293330FC0016204B
:1003F000092A7008053C031D012A3630FC0016202E
:10040000092A7008063C031D092A3930FC00162011
:10041000092A780883120313BF000C203C30FC002B
:100420001620790883120313BF000C2002308312B8
:100430000313400203181F2A3F30FC0016208312CA
:100440000313C00AAB294308A8001A20C3004208BE
:10045000A8001A20C2004508A8001A20C5004408B8
:10046000A8001A20C40042084402C60045084302FE
:1004700003183E2A43084502C7004E2A4308450296
:1004800003184D2AC60343083C3CC300F00145084D
:1004900043070318F00AC7004E2AC7014608A900FF
:1004A0001B20C600BF000C203C30FC00162083122D
:1004B00003134708A9001B20C700BF000C201B30F6
:1004C000FC00162083120313A403240A0319A503B6
:1004D00098292708A5002608A400A001A101442905
:1004E000831203130508033885000000000005107F
:1004F000000000008510000000000800000000005F
:10050000831203138514000000000514000000008E
:100510000800083083120313AA002A08AA03003C2B
:100520000319A02ABA1F962A0514972A051000005D
:1005300085143A0DFE39BA000000000085108D2A9E
:10054000F130831685008312051400008514000025
:10055000030105180130003C0319B12A0130AA003B
:10056000B22AAA018510F0308316850083122A086A
:100570000800F13083160313850083120514083038
:10058000AA002A08AA03003C0319D92A0000000087
:100590004B0DFE39CB008514030105180130003CDA
:1005A0000319D52A0130CB04D72AFE30CB0585109C
:1005B000C12A3B08003C0319DF2A0514E02A051074
:1005C000F0308316850000000000831285140000BF
:1005D000000085104B080800831203133C08003C00
:1005E0000319F42A0515F52A05113D08860085151D
:1005F000000085110614AA0128302A020318022BD4
:10060000AA0AFC2A0800831203133E08F000F00C2B
:10061000F00CF00C700C0F39AA00093C03181A2BCF
:100620000130BC00F00137302A070318F00ABD0082
:100630000A20232B0130BC00F00130302A070318B8
:10064000F00ABD000A200F3083120313BE053E08D6
:10065000093C0318352B0130BC00F00137303E0750
:100660000318F00ABD000A203E2B0130BC00F00147
:1006700030303E070318F00ABD000A20080083123C
:1006800003133F08F000F00CF00CF00C700C0F3965
:10069000AA00F0012A08303E0318F00AC8000D2015
:1006A0000F3083120313BF05F0013F08303E0318DB
:1006B000F00AC9000D20080083120313CC00093092
:1006C000CB000610000000000E20CB0B6A2B061496
:1006D0000E200800CC0C031C6F2B0614642B061094
:1006E000642B263083120313B900B90B752B080055
:1006F00083120313CB01831203134B08F2007B0810
:100700001C20FF39003C0319932B01308312031383
:10071000BC004B08CB0AF2007B081C208312031399
:10072000BD000A207B2B080083120313BC0182301A
:10073000BD000A207A08BE000B2083120313BC01FF
:100740008530BD000A2079081F39BE000B208312B6
:100750000313BC018830BD000A2077083F39BE0072
:100760000B2083120313BC01C030BD000A207608A1
:100770003F39BE000B2083120313BC01C330BD0000
:100780000A2075087F39BE000B2083120313BC01B9
:10079000C630BD000A2074087F39BE000B208312CA
:1007A0000313BC018A30BD000A2078080739F8001D
:1007B000F0007008003C031DE02BFB010F20102C03
:1007C0007008013C031DE82B0330FB000F20102CA8
:1007D0007008023C031DF02B0630FB000F20102C8C
:1007E0007008033C031DF82B0930FB000F20102C70
:1007F0007008043C031D002C0C30FB000F20102C53
:100800007008053C031D082C0F30FB000F20102C36
:100810007008063C031D102C1230FB000F20102C1A
:10082000080083120313CA010620A230BA00082070
:10083000CA000230BA000820CA040620A330BA0059
:100840000820CA04C801063048020318342CBB0132
:100850000920F0004808743E84007008831380006B
:1008600083120313C80A232C0130BB000920FA00AD
:1008700007204A0808000620A230BA000820BA0162
:1008800008202030BA0008201330BA0008203208AF
:10089000BA0008203108BA0008203008BA00082041
:1008A0002E08BA0008202F08BA0008202D08BA0028
:1008B00008202C08BA0008200530BA0008200830AB
:1008C000BA0008200830BA0008200630BA00082014
:1008D0008330BA0008208230BA0008200130BA0004
:1008E0000820BA0108200720080079081F39F900FC
:1008F00078080739F80077083F39F70076083F395C
:10090000F60075087F39F500063083120313CA001C
:100910004A08003C0318D42C2208F1002308F000F8
:10092000F00CF10CF00CF10CF00CF10CF00CF10CE3
:10093000F00CF10CF00CF10CF00CF10C700CF10C53
:100940000039F0007108F101C80023080039F000F7
:100950002208FF39C9000620A030BA000820AB00E9
:100960004808BA000820AB044908BA000820AB04C4
:100970004A08743E84008313000883120313BA00EC
:10098000082007200A30FD001420831203132308D7
:10099000F0000030F0072208013E0318F00AA20020
:1009A0007008A300CA03882C08005E30FE00000017
:1009B0000000000000000000000000000000000037
:1009C0000000000000000000FE0BDA2C0000FD0B10
:1009D000D52C00000800831203132008F100210821
:1009E000F000F00CF10CF00CF10CF00CF10CF00C30
:1009F000F10CF00CF10CF00CF10CF00CF10C700C93
:100A0000F10C0039F0007108F101C900210800392A
:100A1000F0002008FF39CA000620A030BA000820E4
:100A20004908BA0008204A08BA0008200620A13068
:100A3000BA000820C8010530480203182C2DBB015C
:100A40000920F0004808743E840070088313800079
:100A500083120313C80A1B2D0130BB000920F900C3
:100A600007202108F0000030F0072008063E031898
:100A7000F00AA0007008A100080083120313C80147
:100A8000831203134808F2007C081C20FF39003C45
:100A90000319532D831203134808C80AF2007C0877
:100AA0001C200D20402D0800FA30FD001420FA30E3
:100AB000FD001420FA30FD001420FA30FD0014204F
:100AC000FF0B542D0800083083120313C800C9011E
:100AD000051B682D1920051B682D0E20C90CC91394
:100AE000051BC917C80B6D2D0E20490808001330CF
:100AF00083120313B900B90B7B2D08008312031373
:100B0000280E0F39F000700770077007F007F00D1E
:100B1000701028080F397007080083120313290C7E
:100B2000F000700C3F392907F000700C7F3929075D
:100B3000F000700C7F39F000F00C700C3F39290781
:100B4000F000700C7F392907F000700E0F39F000AB
:100B5000F100F10D710DFC397007F100710DFE39D6
:100B60002902F100700EF0397107080005308A0083
:100B7000BE30720703188A0A720882072834533479
:100B800075346E342934003405308A00CC30720755
:100B900003188A0A7208820728344D346F346E3481
:100BA0002934003405308A00DA30720703188A0AC3
:100BB000720882072834543475346534293400347B
:100BC00005308A00E830720703188A0A7208820723
:100BD00028345734653464342934003405308A00AD
:100BE000F630720703188A0A7208820728345434D0
:100BF000683475342934003406308A0004307207B2
:100C000003188A0A72088207283446347234693419
:100C10002934003406308A001230720703188A0A19
:100C20007208820728345334613474342934003410
:100C300006308A002030720703188A0A7208820779
:100C400032343034303430342F34303430342F3484
:100C500030343034283420342034203429342034C3
:100C6000003406308A003930720703188A0A720885
:100C70008207303430343A34303430342E34303427
:100C800030342034203420342034203420342034B4
:100C90002034003406308A005230720703188A0A62
:100CA000720882070D340A34003406308A005D3041
:100CB000720703188A0A7208820783345E34833409
:100CC00043348334803483344A3481345B34833412
:100CD00068340D340A340D340A34003406308A0086
:100CE0007630720703188A0A720882079334FC343C
:100CF0008E34BA348E349E348D348F342034203484
:100D00002034203420342034203420342034203443
:100D1000203420342034203420349134DE348E3496
:100D2000BA348E349E348D348F34203420342034C1
:100D30002034203420342034203420342034203413
:100D400020342034203420348D34DD348E34BA34D1
:100D50008E349E348A34D4340D340A340034063050
:100D60008A00B730720703188A0A720882072F3484
:100D7000003406308A00C130720703188A0A7208EC
:100D8000820728349334FA3429342034003406306E
:100D90008A00CF30720703188A0A72088207283443
:100DA0008C348E3429342034003406308A00DD300F
:100DB000720703188A0A7208820728348934CE34ED
:100DC00029342034003406308A00EB3072070318CF
:100DD0008A0A7208820728349034853429342034F2
:100DE000003406308A00F930720703188A0A720844
:100DF000820728349634D83429342034003407301C
:100E00008A000730720703188A0A7208820728349A
:100E10008B34E03429342034003407308A00153014
:100E2000720703188A0A72088207283493347934C7
:100E300029342034003407308A0023307207031825
:100E40008A0A720882073A34003407308A002D304B
:100E5000720703188A0A720882072034203420346B
:060E6000203420340034B0
:00000001FF
